:1000000000308A00CB2A0000A001A101A201A301B7
:100010008316A001A101A201A30183127D087C0423
:100020007B047A040319622820308316A40003108D
:100030008312F60DF70DF80DF90D8316A00DA10D25
:10004000A20DA30D83127D0883162302031D3828F9
:1000500083127C0883162202031D382883127B0832
:1000600083162102031D382883127A088316200282
:10007000031C592883127A088316A00283127B0876
:10008000031C7B0F442847288316A10283127C0897
:10009000031C7C0F4C284F288316A20283127D0874
:1000A000031C7D0F542857288316A30283120314C0
:1000B00083168312A00DA10DA20DA30D8316A40B10
:1000C000172883120000A0308400003420308316EB
:1000D000A400A001A101A201A30183127908A30039
:1000E0007808A2007708A1007608A0000310201C61
:1000F00095287A088316A00783127B0803187B0FC4
:10010000822885288316A10783127C0803187C0F98
:100110008A288D288316A20783127D0803187D0F75
:10012000922895288316A30783128316A30CA20C8A
:10013000A10CA00C8312A30CA20CA10CA00C831682
:10014000A40BA328A5288312762883128A1180295C
:100150007330840000080319BC280130A100A001FD
:10016000A00BB028A10BAF284A30A000A00BB628E6
:0A01700000000000800BAD280034F1
:100200000130A3000A30FE0023088A007B08073A69
:100210000739820700000000000000000000000015
:1002200000000000FC0CFB0CFC0CFB0CFC0CFB0CA1
:100230001F30FC057C08FD00FB0A0319FC0AFD0ABF
:10024000000000000000FB0B2629FD0B20290034D4
:0E025200F208031D4029F308031D4029F4089B
:10026000031D3529F50803193F290330FC00E83048
:10027000FB00002174080319F503F4032F29C92991
:10028000F9010730F800A130F7002030F600FD0139
:10029000FC017308FB007208FA0004202308F9002F
:1002A0002208F8002108F7002008F60048307602FE
:1002B000A9007708AA000030031C0130AA027808C0
:1002C000AB000030031C0130AB027908AC000030F9
:1002D000031C0130AC02A801A7017508A600740830
:1002E000A5002808F9002708F8002608F7002508C7
:1002F000F600FD01FC017308FB007208FA00662895
:100300002308A8002208A7002108A6002008A500AD
:100310002808F9002708F8002608F7002508F60045
:10032000FD01FC010130FB00F430FA000420230839
:10033000A8002208A7002108A6002008A50026087A
:10034000F8002508F700F708031DA929F808031984
:10035000C9297618AD290611AE290615831606118E
:100360008312761CB5298611B62986158316861147
:1003700001308312F6062A08FA002908F9002A0833
:10038000FC002908FB00002177080319F803F70394
:10039000A329003444164408831687008312071EDD
:1003A000C92AF430F100F3017108F200F50132308E
:1003B000F40029216430F107D3290430F200FA3027
:1003C000F300A820F20BDF2983160613831206130D
:1003D000831686138312861383160612831206125F
:1003E000831686128312861283160612831206164D
:1003F00083168612831286120430F200FA30F3005C
:10040000A820F20BFE298316061283120612831609
:100410008612831286120430F200FA30F300A8200C
:10042000F20B0D2A83168612831286168316061285
:10043000831206120430F200FA30F300A820F20B07
:100440001C2A831606128312061283168612831242
:1004500086120430F200FA30F300A820F20B2B2AA7
:1004600083160613831206178316861383128613C8
:100470000430F200FA30F300A820F20B3A2A831677
:100480000613831206138316861383128613043011
:10049000F200FA30F300A820F20B492A83168613E3
:1004A0008312861783160613831206130430F20094
:1004B000FA30F300A820F20B582A83160613831291
:1004C000061383168613831286130430F200FA3063
:1004D000F300A820F20B672A83160613831206176F
:1004E000831686138312861383160612831206164A
:1004F00083168612831286120430F200FA30F3005B
:10050000A820F20B7E2A8316061383120613831685
:10051000861383128613831606128312061283161D
:100520008612831286120430F200FA30F300A820FB
:10053000F20B952A831686138312861783160613E9
:1005400083120613831686128312861683160612EA
:10055000831206120430F200FA30F300A820F20BE6
:10056000AC2A83160613831206138316861383128E
:1005700086138316061283120612831686128312BE
:1005800086120430F200FA30F300A820F20BC32ADE
:10059000CA298A11F02A84011F3083050730831687
:1005A0009F0082308312AD009830AE00AF00403023
:1005B000B000B100B2006030B3008630B400B43097
:1005C000B5006030B600A430B700B800B9006130A3
:1005D000BA000330BB00F030BC00FF30C400CA29B1
:1005E0000230F3008030F200F501C830F400292118
:1005F0003230F300A8200230F3008030F200F50121
:10060000C830F4002921043083169F0083121F088C
:10061000383901389F000430F100FA30F300A82087
:10062000F10B0D2B0130ED000230EE00EF018316CF
:1006300006138312061783168613831286138316F6
:10064000061283120616831686128312861208304B
:10065000A1001F08C73921049F00000000001F15DA
:100660001F19302B1E08313C031C4A2BEF010130AF
:10067000EE00831606138312061783168613831261
:1006800086138316061283120616831686128312A9
:100690008612272B0030A1001F08C73921049F00B4
:1006A000000000001F151F19532B1E08313C031CAE
:1006B0006C2BEF01EE0183160613831206178316C7
:1006C0008613831286138316061283120616831668
:1006D000861283128612272BEF08031DBF2B831669
:1006E000061383120613831686138312861383164A
:1006F000061283120612831686128312861283163E
:100700008613831286178316061383120613831625
:10071000861283128616831606128312061214306E
:10072000F300A8208316061383120613831686137C
:1007300083128613831606128312061283168612FC
:1007400083128612C830F300A820EE08031DB12BD7
:1007500083160612831206168316861283128612D9
:10076000ED016E0BBD2B831606138312061783163D
:100770008613831286130130ED00EF0A272B272BF7
:02078000630014
:02400E00793FF8
:00000001FF
